:020000040000FA
:02000000CF2A05
:08000800A500260EA6008312DC
:100010008C011A0880000A3A031924167F30040262
:10002000031C840A260E8300A50E250E09008A01F2
:100030000F3982073F3406345B344F3466346D34F5
:100040007D3407347F346F3400340034003400349E
:10005000003400341530350203181D34350882078A
:100060001A341A341A341A341A341A341A34193421
:100070001E341D341C341B3419341F341E341D34FB
:100080001B341A3419341F341D341530350203184B
:100090001D34350882071D341D341D341D341D34B4
:1000A0001D341D341C341A3419341F341E341C34CE
:1000B0001B341A3419341E341D341C341B341934C7
:1000C00036038207033403346E28043404340434C2
:1000D0000434043404347328033403342A203702EC
:1000E000031C0334043445203702031C0434033456
:1000F000310382071F3486281F341E341F341E34F8
:100100001F341F341E341F341E341F34300803398B
:10011000031D1C341D3436038207093408340734A8
:100120000634053405340534053406340734083400
:10013000093436038207113412341334143415345D
:100140001534153415341434133412341134A419FD
:1001500002348B20FE3E3802031C02348B20013E09
:100160003802031C01349920023E3802031802347D
:100170009920FF3E38020318013400342708820713
:10018000602A572A532A512A27088207732A6F2A7E
:10019000662A642A270882074C2A482A442A3A2ACF
:1001A0002D088207102A122A152A182A2D088207DC
:0A01B0001A2A1C2A1F2A222A322ACA
:10020000A000A1010A302002031C0800A000A10ADE
:1002100002290F39A000A007A00DA00DA007A0077C
:10022000080024128B130D306406031DA529243009
:100230004006031DA52947304106031DA52950305E
:100240004206031DA5295A304306031DA529443043
:100250004406031DA52941304506031DA529510863
:10026000092152080F39A0070319A52920302002BF
:100270000318A5292008B2005408092155080F3990
:10028000A0070319A5290D3020020318A52920086D
:10029000B10032305706031DA52930305806031D22
:1002A000A529590809215A080F39A007073020024B
:1002B000031CA529153020020318A5292008B00029
:1002C0004708092148080F39A007183020020318F1
:1002D000A5292008B3006020B307003E1830330280
:1002E000031C8029B300B20A78203202031C802943
:1002F0000130B200B10A0D30310201300318B100F3
:10030000490809214A080F39A0073C302002031888
:10031000A5292008B4004B0809214C080F39A00773
:100320003C3020020318A5292008BA003408B9007F
:100330003308B8003208B7003108B6003008B500FD
:10034000A414AD010430A406A90A8B13831620302F
:1003500098001930990020308C0083121A089030D0
:10036000980040308400C0308B0008000310851ACC
:1003700003140800A2000000BD29BE29A20BBB295E
:1003800064000800A41200306500FF30BA2120305C
:100390006500FF30A100B621CD29CE29031CD32949
:1003A000A10BCB29DC29FF30A100B621D729D82900
:1003B00003180800A10BD529A4160800A0000830D6
:1003C000A10000306500A00C0318EE2900002730C2
:1003D000BA21203065000330BA21F5290330BA2153
:1003E000203065002730BA21F5290330BA21A10B4E
:1003F000E1290800A3010830A100003065000330A6
:10040000BA21203065000730BA210714B621071041
:10041000A30CB621031C092AA10BFD2923080800FF
:10042000AD0AC229AD0ACC30DE29AD0A4430DE293E
:10043000A4100800AD0AC229AD0ACC30DE29AD0AED
:10044000BE30DE29AD0AFA21AC002410AC1B241406
:10045000AC0C3F30AC05241C08003F30AC06AC0AA5
:10046000AC050800A4100800AB01A91DBE28291D79
:10047000C428CA280830AA002C0803190800C03074
:1004800024184030AB0008000430AA002C087E2A53
:100490000230AA002C08812A0130AA006330AB0088
:1004A00008003808772A0430AA003808812A023068
:1004B000AA0039080021210817200138AB000800E4
:1004C0000130AA003908812A37087E2A0430AA00A0
:1004D00037080021200817200138AB00080002303F
:1004E000AA0036087E2A0130AA003608812A002197
:1004F0000830AA00210803190800832A00212108D6
:10050000832A002120081720AB0008002030840037
:100510008001840A041F882A84010C30B80022302C
:10052000B9000530B6000630B7000830B500083015
:10053000AC0000308500AA0000308600AB004030DF
:10054000870008000B1DA22A850186010630810064
:100550000B116400033062008B138316203085007A
:10056000003086008630870007309F0083128B178B
:100570002C08A720003A0319C62A013A031DC32AF2
:10058000281CC62AC52A2808031DAB012A08850095
:100590002B08860008008622A622A5210800CB226F
:1005A000A222A41CD72A2419D020241DD620241A24
:1005B00011218B1334228B17A70A271DD02AA701DC
:1005C000A80A0330A8058718E92AA415FA30AE0056
:0A05D000D02AAE030319A411D02AAB
:02400E00363F3B
:00000001FF
